:103FC5000ECF0EBB0EA70E920E7C0E650E4D0E3457
:103FD5000E190DFE0DE10DC40DA50D850D640D42E7
:103FE5000D1E0CFA0CD40CAE0C860C5D0C330C08B3
:103FF5000BDC0BB00B820B540B250AF50AC40A9394
:104005000A610A2F09FD09CA09960963092F08FCE7
:1040150008C808950861082E07FB07C807960764B6
:104025000733070206D206A206730645061705EAF8
:1040350005BF059305690540051704F004C904A3E8
:10404500047E045A0437041503F403D303B403961A
:104055000378035B033F0324030A02F002D702BF80
:1040650002A80292027C02670253023F022C021A46
:10407500020801F701E601D601C701B801A9019CB3
:10408500018E018101740168015D01510146013C08
:1040950001320128011F0115010D010400FC00F486
:1040A50000EC00E500DE00D700D000CA00C300BD6B
:1040B50000B800B200AD00A700A2009E00990094D0
:1040C5000090008C008700840080007C00780075DB
:1040D5000072006E006B0068006500620060005DA4
:1040E500005A0058005500530051004E004C004A3C
:1040F50000480046004400430041003F003E003CAC
:10410500003A0039003700360035003300320031FF
:10411500002F002E002D002C002B002A002900283E
:104125000027002600250024002300010C010105BD
:1041350002011E030A9604013205050506006407FF
:10414500010108000009015A0E01010F00011200CA
:104155006413010114013C1501FA1664FA17FFFFF7
:104165001D00072000072400022701012F013C3014
:10417500030332010335FFFF3603073CFFFF3DFF15
:10418500FF180002191E461A00021B00022D32C834
:104195002E0001FAFAFA18000019FFFF1A00001B99
:1041A50000002D32C82E0001FAFAFA18000019FF96
:1041B500FF1A00001B00002DFFFF2EFFFFFAFAFA81
:10004800900787E0FEA3E0FF7457BE0010D39F40DF
:100058000C90412F12001EE493F599804C900014E7
:10006800E0D394044014900787E0FEA3E0FF90419A
:100078002F12001EE493F599802F900014E0D3947A
:10008800034014900787E0FEA3E0FF90414412006C
:100098001EE493F5998012900787E0FEA3E0FF9095
:1000A800415912001EE493F59990078712000E90AB
:1000B8000787E0FEA3E0FF746C6F4E7003751300B2
:1000C80022900073E0B402087401900073F0D20E1D
:1000D80090013BE090002AF090013CE090002BF06A
:1000E80090013DE090002CF0A20AB3401690013B2D
:1000F800E0700C90013CE0700690013DE0600280E9
:1001080002C20A90013BE0B4300F90013CE0B447D2
:100118000890013DE0643B60028004D20B8002C27B
:100128000BE558B40102800302024B900058E0F539
:1001380066900063E0F568900064E0F569900075EA
:10014800E0F56A90007BE0900029F090007DE0F5F2
:100158006590007EE0F567900081E0F5649000828C
:10016800E0F563900091E0900041F0900092E090FB
:100178000042F0900093E0900043F0900094E090EB
:100188000044F0900095E0900045F0900096E090D3
:100198000046F0900097E0900047F0900098E090BB
:1001A8000048F090009AE0900033F090009BE090B7
:1001B8000034F090009CE0900035F090009DE090B5
:1001C8000036F090007AE0B4011790000A740FF03E
:1001D800A374FFF090000CE4F0A3F0740290007A8E
:1001E800F090007AE0B4035990000CE0FEA3E0FF21
:1001F80090000AE0FCA3E0FD1200037410124325EE
:100208007408124317EF900026F0EF700674FF9001
:100218000026F0740090007AF090000BE090002720
:10022800F090000AE0900028F0900026E090078AFD
:10023800F0900027E090078BF0900028E090078C62
:10024800F0803F900082E07006755801756300A247
:100258000AB3402E90013BE090002AF090013CE068
:1002680090002BF090013DE090002CF090002AE0E7
:10027800700C90002BE0700690002CE06002800269
:10028800C20AE5667003756602E568700375680260
:100298007E897FE7E5668E048F05FF1243078C3958
:1002A8008D3AE56975F0FAA4FFAEF0E5688E048F23
:1002B80005FF1243078C3D8D3E900050E0F560909D
:1002C800004DE0FE90006AE0B5061890004CE0FE94
:1002D800900069E0B5060C90004BE0FE90005AE0F3
:1002E8006E606F90006AE07006900069E0600674C6
:1002F8000090005AF090006AE0B402089000497437
:1003080001F08005900049E4F0900069E0B402082B
:1003180090004A7401F0800590004AE4F09000696A
:10032800E0600690004AE060028005756004800382
:10033800756005E559B55802D20E900069E0900045
:100348004CF090006AE090004DF090005AE0900068
:100358004BF0740190009FF074009000A0F07400BE
:100368009000A1F074009000A2F074019000A3F036
:1003780074009000A4F074009000A5F0740190003F
:10038800A6F074009000A7F074009000A8F0740024
:100398009000A9F074019000AAF074009000ABF0EE
:1003A80074009000ACF074019000ADF074009000FF
:1003B800AEF074009000AFF074009000B0F07401DB
:1003C8009000B1F074009000B2F074009000B3F0A7
:1003D8007401900363F07400900364F07400900358
:1003E80065F07400900366F07401900367F0740080
:1003F800900368F07400900369F074019003A3F00F
:1004080074019003A4F074009003A5F074009003A5
:10041800A6F074019003A7F074009003A8F074008C
:100428009003A9F074009003E3F074019003E4F0E2
:1004380074009003E5F074009003E6F074019003F3
:10044800E7F074009003E8F074009003E9F074009A
:10045800900423F07400900424F07400900425F0B4
:100468007400900426F07401900427F0740090043E
:1004780028F07400900429F07400900463F074006C
:10048800900464F07401900465F07401900466F0BF
:100498007400900467F07400900468F0740090048D
:1004A80069F022E5B554F7F5B5E5B554FDF5B5C2E3
:1004B80093C294C291C292756F00757000C287C2D0
:1004C80007E5B554FBF5B5755105E55104F55290AE
:1004D8000050E0F560900025E4F0C209E5B554FE4F
:1004E800F5B590004EE4F022750A00750900AE09D2
:1004F800AF0A7457BE00039F50030205AD90412F09
:1005080012001EE49390004F12433D0FBF00010EEE
:10051800E0FC90412F12001EECFEE493FFEEC39F17
:100528005026AE09AF0A0FBF00010E90412F1200EE
:100538001EAE09AF0AE493FC90412F12001EE4930B
:1005480090004F12433DECF0AE09AF0A90412F12D4
:10055800001EE49390004F12433DE0FC904131129D
:10056800001EECFCE493FDECD39D40199041311240
:10057800001EE493FC90412F12001EE49390004F5C
:1005880012433DECF0AE09AF0A74022FFF50010E82
:100598008E098F0A780A740126F6500418E436F694
:1005A80040030204F622750A00750900AE09AF0A75
:1005B8007415BE00039F500302067B90418612000B
:1005C8001EE49390004F12433D0FBF00010EE0FC64
:1005D80090418612001EECFEE493FFEEC39F502666
:1005E800AE09AF0A0FBF00010E90418612001EAE81
:1005F80009AF0AE493FC90418612001EE493900030
:100608004F12433DECF0AE09AF0A90418612001E2E
:10061800E49390004F12433DE0FC90418812001E85
:10062800ECFCE493FDECD39D401990418812001E28
:10063800E493FC90418612001EE49390004F12430D
:100648003DECF0AE09AF0A740F6F4E7006750A15CF
:10065800750900AE09AF0A74022FFF50010E8E090A
:100668008F0A780A740126F6500418E436F6400317
:100678000205B422750A00750900AE09AF0A74159F
:10068800BE00039F500302074990419B12001EE4DD
:100698009390004F12433D0FBF00010EE0FC9041C4
:1006A8009B12001EECFEE493FFEEC39F5026AE099A
:1006B800AF0A0FBF00010E90419B12001EAE09AF9A
:1006C8000AE493FC90419B12001EE49390004F12A1
:1006D800433DECF0AE09AF0A90419B12001EE49333
:1006E80090004F12433DE0FC90419D12001EECFC2F
:1006F800E493FDECD39D401990419D12001EE493B4
:10070800FC90419B12001EE49390004F12433DEC75
:10071800F0AE09AF0A740F6F4E7006750A157509A9
:1007280000AE09AF0A74022FFF50010E8E098F0A1E
:10073800780A740126F6500418E436F640030206D7
:100748008222750A00750900AE09AF0A7415BE0049
:10075800039F50030208179041B012001EE49390C3
:10076800004F12433D0FBF00010EE0FC9041B01254
:10077800001EECFEE493FFEEC39F5026AE09AF0ABD
:100788000FBF00010E9041B012001EAE09AF0AE47F
:1007980093FC9041B012001EE49390004F12433D29
:1007A800ECF0AE09AF0A9041B012001EE49390003D
:1007B8004F12433DE0FC9041B212001EECFCE49362
:1007C800FDECD39D40199041B212001EE493FC90B9
:1007D80041B012001EE49390004F12433DECF0AE7E
:1007E80009AF0A740F6F4E7006750A15750900AEC9
:1007F80009AF0A74022FFF50010E8E098F0A780A7A
:10080800740126F6500418E436F640030207502215
:10081800054D22054C22054EC2CF2290F800E493E4
:100828006406600280FE75840175A70075FF8090DC
:100838000789E4F075C91075A70F75A1C775A700DA
:1008480075D90075CEFF75A70F75F1FE75F2FF75A6
:10085800F33775F47875A4BA75A5FF75A60775AE54
:100868000075AFFF75D48175D5FF75D6FF75D7FFB5
:10087800C296C295C2A0E5B554EFF5B5E5B554DF0B
:10088800F5B5E5B554F7F5B5E5B554FDF5B575A776
:100898000075A20175A14775F80975BC0175BE04FC
:1008A80075BD6C75BE0775BDA075BE0875BD0175B3
:1008B800BC0075BB1875BC2075BA0875E88075D181
:1008C8001375A70F75E10575E20075C740759700A8
:1008D800759780740A1242F77597C0E5975420708F
:1008E8000280F8758F0275A700D2AF75980075A9B8
:1008F8000C75A70F75AB4375ADFB75AC1E75A700DE
:10090800758911758E00758C00758A00D2A9D28CF4
:10091800758D00758B00D2ABD28E75CD0075CC006D
:1009280075CA0075CB00D2ADC2CFD2CA7591047515
:1009380092007593CD75EF0675D94075CF01900774
:1009480087E4F0A3F0751300751400C299D20A74F5
:10095800C8F5187517001228EE75A70FE5FB90006B
:100968001AF0E5FA90001BF0E5F990001CF075A765
:100978000090F800E493F508122A25122F5F9007DB
:100988008AE0900026F090078BE0900027F090070F
:100998008CE0900028F090078DE0900029F09007F7
:1009A8008EE0F56690078FE0F568900790E0F569AE
:1009B800900791E0F56A900792E0F565900793E05B
:1009C800F567900794E0F564900795E0F563900764
:1009D80096E090002AF0900797E090002BF090079F
:1009E80098E090002CF0900799E0900041F0900773
:1009F8009AE0900042F090079BE0900043F0900747
:100A08009CE0900044F090079DE0900045F090072E
:100A18009EE0900046F090079FE0900047F0900716
:100A2800A0E0900048F09007A1E0900033F0900714
:100A3800A2E0900034F09007A3E0900035F0900712
:100A4800A4E0900036F07400900083F090013BE041
:100A5800700C90013CE0700690013DE0600280045B
:100A6800C20A8002D20A90F807E493900021F0901D
:100A78000021E0440A900021F0900021E054FE900B
:100A88000021F07406900012F07402900013F090A8
:100A9800F802E493900014F07403900015F07403C6
:100AA800900016F07405900017F07405900018F087
:100AB800900014E0B404067404900018F090001438
:100AC800E0B403067403900018F07404900019F061
:100AD80090F804E49390001DF0740090001EF090CC
:100AE800F805E49390001FF090F806E49390002036
:100AF800F074FF900022F07441900126F074699020
:100B08000127F07473900128F07469900129F0743A
:100B18006E90012AF0742090012BF0744190012C02
:100B2800F0743790012DF0743590012EF0743090E8
:100B3800012FF07445900130F07420900131F07469
:100B480035900132F07453900133F0747090013491
:100B5800F090007BE0D394014006740090007BF095
:100B6800755801755901740390004CF01200C912B0
:100B780004F0900014E0B4040512067C8011900083
:100B880014E0D3940440051205AE800312074A12FC
:100B9800291AE5B554FEF5B5900025E4F0900787CD
:100BA800E4F0A3F0752400752300754800752A0049
:100BB800752900754900753200753100754A007550
:100BC8005400755500755A007551057552017534F4
:100BD8003C7533007572007571007573CD755600DC
:100BE80075570075430075440075450075460075D6
:100BF8005B00754700754200754100900006E4F0FF
:100C0800A3F0900008E4F0A3F0755E00755F009013
:100C1800000E74FDF0A374E8F0900023E4F074640F
:100C2800900024F0C200D201C202D203754D0075B3
:100C38006D00E5B554BFF5B5E5B5547FF5B5C2A16E
:100C4800C2A2C297C20E7E017F00900028E0124324
:100C580025900027E02FFF50010E90000AEEF0A328
:100C6800EFF0900026E0700674FF900026F09000E8
:100C78000AE0FEA3E0FFEFD394FFEE940F40079045
:100C8800000AE4F0A3F07400900072F07400900081
:100C98007AF07400900083F0740090008EF0740075
:100CA8009000B5F0E5677003756704743A90074FD4
:100CB800F074FD900750F0900415E0900455F0D2C0
:100CC800B0D2B7D2A7D2A6D2B1D2A3C207A2B6B326
:100CD8009204A2B3B39205D29CD2EC75CF01A2982C
:100CE800B34005C2981232C3E5136006A299B3B3A4
:100CF80040028005C299123839E51464016005E59F
:100D080014B4040280D5E54DD39405400CE55AC3CC
:100D180094C85002055A754D00E573C394F0501AF3
:100D2800787112003FAE71AF72EFD394E8EE94037E
:100D380040080573757200757100C28E7E047F00CD
:100D4800E54C124325E58D75F004A4FDACF0EF2DBC
:100D5800FDEE3CFCE58B75F04084FF7E00ED2FFF37
:100D6800EC3EFE8E258F26D28EA2B6300401B350FB
:100D780003020EB9A2B6300401B35003020EB9A2A1
:100D8800B6405A0554E5B54401F5B5900024E4F0A1
:100D9800E554D3956640447C897DE71241C58E238E
:100DA8008F24E5482FFF50010E74011243178E233C
:100DB8008F24852448755401C28E758D00758B006B
:100DC800754C00D28E7403BE00039F500690002518
:100DD8007401F0E543B40603754300D204A2B6B328
:100DE8005003020EB9C20490006CE0601812397A00
:100DF800A200B34008E5B54408F5B58006E5B5544A
:100E0800F7F5B58002C20090006FE06018123ACF83
:100E1800A202B34008E5B54402F5B58006E5B5542D
:100E2800FDF5B58006E5B554FDF5B5A207B3400854
:100E3800E5B54440F5B58006E5B554BFF5B5900075
:100E48005AE06008E5B54480F5B58006E5B5547FFD
:100E5800F5B590004AE0B40104D2A18002C2A19085
:100E68000049E0B40104D2A28002C2A2A209B340A0
:100E780004D2978002C297900018E0FE900014E018
:100E8800C39E4009900014E0D39408400974FB9075
:100E98000023F01204AB90001DE0601590001DE0E7
:100EA800FE900017E06E600974FE900023F01204B3
:100EB800ABC2CA7E017F00E54E124325E5CD2FFF68
:100EC80050010E8E278F28D2CAE565B401489000DC
:100ED8000EE0FCA3E0FDEFC39DEE9C4039B208E5AF
:100EE8002A45296013A208B34008E5B54404F5B5BE
:100EF8008006E5B554FBF5B590000EE0FEA3E0FFD3
:100F0800900010E0FCA3E0FDEF2DFDEE3CFC90000E
:100F18000EECF0A3EDF0A2B3300501B35003020FBD
:100F2800FEA2B3300501B35003020FFEA2B3500373
:100F3800020FF70555E5B54401F5B5900024E4F036
:100F4800E555D395685003020FF57CEA7D60AE271E
:100F5800AF281241C58E298F2AE56912432574FFEF
:100F68008E048F05FF1243078C298D2AE5492DFD34
:100F780050010C74018C068D071243178E298F2A95
:100F8800852A49A209B34015746412432590006864
:100F9800E08E048F05FF1243078C298D2A755501B1
:100FA80090000EE0FEA3E0FFAC27AD2812000390EE
:100FB800000EEEF0A3EFF0E567FF124307740AFF97
:100FC80012430790007CE08C068D071243257414A9
:100FD8008E048F05FF124307900010ECF0A3EDF08C
:100FE800C2CA75CD0075CC00754E00D2CAD205A212
:100FF800B3B34002C205900025E0B40107E556C32B
:101008009406400302161EE56D9028CDF828287333
:1010180090005AE0C39402400302116CE551D39446
:1010280001500302116CE55175F040A4FFAEF09039
:10103800031312001EE0C395455018E55175F040A2
:10104800A4FFAEF090031212001EE0F52E752D00DD
:1010580002116CE55175F040A4FFAEF09003111237
:10106800001EE0C395454003021108E55175F040A4
:10107800A4FFAEF090031212001EE55175F040A4D3
:10108800FFAEF0E0FC90031012001EECFEE0FFEE55
:10109800C39FFEE5518E0475F040A4FFAEF09003A7
:1010A8001112001EE0F40425458C0088F0A4FFAE60
:1010B800F0E5518F048E0575F040A4FFAEF0900363
:1010C8001312001EE55175F040A4FFAEF0E0FA904F
:1010D800031112001EEAFEE0FFEEC39FFECDCCCD49
:1010E8008E07124307E55175F040A4FFAEF0900358
:1010F8001012001EE02DFD50010C8C2D8D2E8064E9
:10110800E55175F040A4FFAEF090031012001EE503
:101118005175F040A4FFAEF0E0FC90030F12001EE2
:10112800ECFEE0FFEEC39F8545F0A4FFAEF0E5516D
:101138008F048E0575F040A4FFAEF09003111200E5
:101148001EE0FECDCCCD8E07124307E55175F04069
:10115800A4FFAEF090030F12001EE02DFD50010C0D
:101168008C2D8D2E756D0102161E90005AE0C394C9
:10117800024003021320900050E0D395515003021F
:1011880012C8E55175F040A4FFAEF09003191200A3
:101198001EE0C395455018E55175F040A4FFAEF028
:1011A80090031812001EE0F52C752B000212C8E5FA
:1011B8005175F040A4FFAEF090031712001EE0C373
:1011C80095454003021264E55175F040A4FFAEF066
:1011D80090031812001EE55175F040A4FFAEF0E030
:1011E800FC90031612001EECFEE0FFEEC39FFEE526
:1011F800518E0475F040A4FFAEF090031712001E44
:10120800E0F40425458C0088F0A4FFAEF0E5518F8A
:10121800048E0575F040A4FFAEF090031912001E6D
:10122800E55175F040A4FFAEF0E0FA900317120004
:101238001EEAFEE0FFEEC39FFECDCCCD8E07124323
:1012480007E55175F040A4FFAEF090031612001E9A
:10125800E02DFD50010C8C2B8D2C8064E55175F030
:1012680040A4FFAEF090031612001EE55175F04041
:10127800A4FFAEF0E0FC90031512001EECFEE0FFA8
:10128800EEC39F8545F0A4FFAEF0E5518F048E05AF
:1012980075F040A4FFAEF090031712001EE0FECDDB
:1012A800CCCD8E07124307E55175F040A4FFAEF090
:1012B80090031512001EE02DFD50010C8C2B8D2C77
:1012C800E551B40123E560D39401401CE55604D3ED
:1012D80095514014E545C39405500D900360E0A86E
:1012E80029B80006952A40028003755102E551B5D8
:1012F8006022900050E0D395514019E55175F040B7
:10130800A4FFAEF090031812001EE0A823B8000650
:101318009524400280020560756D0202161E900039
:101328005AE0B4022AE55175F040A4FFAEF09003EC
:101338001812001EE0F52C752B00E55175F040A43D
:10134800FFAEF090030F12001EE0F52E752D0090F1
:10135800005AE0B4030F900052E0F52C752B00758D
:101368002E00752D00756D0302161EE55175F040AF
:10137800A4FFAEF090032112001EE0C3955A40036B
:10138800021448900049E07036E551D39401402991
:10139800AE23AF24AC2DAD2EEDD39FEC9E401AE5C5
:1013A8005175F040A4FFAEF090031F12001EE0A894
:1013B80029B80005D3952A5002800215518034E5DA
:1013C80051D394024029AE23AF24AC2DAD2EEDD3DA
:1013D8009FEC9E401AE55175F040A4FFAEF09003D3
:1013E8001F12001EE0A829B80005D3952A500280D4
:1013F800021551E551B55237E551C395605030E5B6
:101408005604D395514028AE23AF24AC2BAD2CEF16
:10141800D39DEE9C4019E55175F040A4FFAEF090C5
:10142800032012001EE0A829B80006952A40028071
:10143800020551C287E55165526005C207755A0019
:10144800756D0402161EE55175F040A4FFAEF090CC
:10145800031B12001EE0B40117E55175F040A4FF0C
:10146800AEF090032112001EE0240AC3955A4003EF
:1014780002151E753064752F00A207B3500B90003B
:1014880061E02405C39545400302151EE55175F03A
:1014980040A4FFAEF090031E12001EE0C395454025
:1014A80064E55175F040A4FFAEF090031D12001ED4
:1014B800E55175F040A4FFAEF0E0FC90031C12006B
:1014C8001EECFEE0FFEEC39F8545F0A4FFAEF0E5FD
:1014D800518F048E0575F040A4FFAEF090031E12E4
:1014E800001EE0FECDCCCD8E07124307E55175F006
:1014F80040A4FFAEF090031C12001EE02DFD500129
:101508000C8C2F8D30AE23AF24AC2FAD30EFD39D94
:10151800EE9C4002D207756D0502161EE551B40116
:101528000990005AE0C3940240030215F29003594F
:10153800E0D3954550030215F2900357E0C3954553
:101548005040900358E0FE900356E0F4042EFE90BD
:101558000357E0F40425458E0088F0A4FFAEF09010
:101568000359E0FC900357E0F4042C8E048F05FF28
:10157800124307900356E02DFD50010C8C2B8D2C47
:10158800802C900356E0FE900355E0F4042E854528
:10159800F0A4FFAEF0900357E08E048F05FF1243CE
:1015A80007900355E02DFD50010C8C2B8D2CE55137
:1015B800C395605030E55604D395514028AE23AF0B
:1015C80024AC2BAD2CEFD39DEE9C4019E55175F062
:1015D80040A4FFAEF090032012001EE0A829B80036
:1015E80006952A40028003755102900049E0B40133
:1015F80006E551640160028003755102E5516552A8
:101608006005C207755A00E55AD3940A4005900050
:061618004EE4F0756D00C8
:1028CD0002101802117202132602137302144E0223
:0228DD001524C0
:10161E00900051E02402A823B80007D3952440027D
:10162E00C207900025E0B4010990005AE0C394036C
:10163E0040030217B2900049E060030216FBE55129
:10164E00D39401403A90004EE07034E55175F0406D
:10165E00A4FFAEF090031512001EE0A823B8001FE1
:10166E00D39524401AE55175F040A4FFAEF09003D7
:10167E002012001EE0A829B80005D3952A5002803A
:10168E00021551E551D39401402FE55175F040A458
:10169E00FFAEF090031312001EE0C39545501AE5FD
:1016AE005175F040A4FFAEF090031F12001EE0A88B
:1016BE0029B80005D3952A500280021551E551D361
:1016CE0094014022E55604C39551501AE55175F028
:1016DE0040A4FFAEF090031F12001EE0A829B80030
:1016EE0005D3952A5002800215510217A7E551D352
:1016FE009402403A90004EE07034E55175F040A4EB
:10170E00FFAEF090031512001EE0A823B8001FD301
:10171E009524401AE55175F040A4FFAEF0900320D9
:10172E0012001EE0A829B80005D3952A50028002A7
:10173E001551E551D39402402FE55175F040A4FFA9
:10174E00AEF090031312001EE0C39545501AE551FA
:10175E0075F040A4FFAEF090031F12001EE0A82902
:10176E00B80005D3952A500280021551E551D39445
:10177E00024022E55604C39551501AE55175F040CA
:10178E00A4FFAEF090031F12001EE0A829B80005BA
:10179E00D3952A500280021551E55165526005C25B
:1017AE0007755A00900061E0D39545500990005599
:1017BE00E0C395455002C20790005AE07003021A2A
:1017CE002DA2A5B34008A2A4B34003021A16AE354B
:1017DE00AF367441D39F749C9E4005783512003FFE
:1017EE00AE35AF36EFB48806EEB41302800302199D
:1017FE00F3A2A550030218A990005AE0B40110906C
:10180E000050E0D3956040020560E55104F552901A
:10181E00005AE0B40256E55175F040A4FFAEF090C8
:10182E00032112001EE0C3955A5041900050E0D3A0
:10183E0095514021E55604D395514019E55175F067
:10184E0040A4FFAEF090031512001EE0A823B800CE
:10185E00069524400280020551855160E55165527E
:10186E006005C207755A00E55104F55290005AE022
:10187E00B40328900050E0D395514008E55604D3A8
:10188E009551500280020551855160E551655260B7
:10189E0005C207755A00E55104F552A2A450030281
:1018AE0019F390005AE0B40173900049E0703AE5E4
:1018BE0051D394014029E55175F040A4FFAEF0904C
:1018CE00031F12001EE0A829B8000FD3952A400A64
:1018DE001551755A008551608003855160800375DE
:1018EE006001E55104F5528033E551D3940240294D
:1018FE00E55175F040A4FFAEF090031F12001EE0FC
:10190E00A829B8000FD3952A400A1551755A00859B
:10191E0051608003855160800375600290005AE02B
:10192E00D3940150030219E7E55175F040A4FFAEC0
:10193E00F090032112001EE0C3955A40030219E7EE
:10194E00900049E07041E551D394014034E5517562
:10195E00F040A4FFAEF090031212001EE0A823B8D0
:10196E00001FD39524401AE55175F040A4FFAEF048
:10197E0090031F12001EE0A829B80005D3952A5027
:10198E000280021551803FE551D394024034E55157
:10199E0075F040A4FFAEF090031212001EE0A823D3
:1019AE00B8001FD39524401AE55175F040A4FFAE40
:1019BE00F090031F12001EE0A829B80005D3952A47
:1019CE00500280021551855160E55165526005C285
:1019DE0007755A00E55104F552E556B40704055E45
:1019EE008003755E00E563B4010EAE35AF36EF646D
:1019FE00407005EE649C6002800EA2A540037558EF
:101A0E0001A2A44003755802A2A5B3B35006A2A426
:101A1E00B3B340028006753600753500021B1BA25B
:101A2E00A5B34008A2A4B34003021B07AE35AF36E0
:101A3E007441D39F749C9E4005783512003FAE359D
:101A4E00AF36EFB48806EEB413028003021B07A272
:101A5E00A5406F900069E0605A90004AE0B401071B
:101A6E0090004AE4F0800690004A7401F090004A1B
:101A7E00E07005756004800375600590004AE0B45F
:101A8E000104D2A18002C2A1E551B4051AE5517537
:101A9E00F040A4FFAEF090031F12001EE0A829B87C
:101AAE000005D3952A50028008755104C207755A55
:101ABE00008003756005E556B40704055E80037566
:101ACE005E00A2A4403390006AE06021900049E0DD
:101ADE00B40107900049E4F080069000497401F0CB
:101AEE00900049E0B40104D2A28002C2A2E556B42D
:101AFE000704055E8003755E00A2A5B3B35006A26F
:101B0E00A4B3B340028006753600753500E55865FE
:101B1E00596006900083E06003021CA3C29C7514FA
:101B2E0000751300C2CAE5589028DFF82828738084
:101B3E0012122F5F800D123038800812311180037F
:031B4E001231EA67
:0F28DF00021B3D021B3F021B44021B49021B4E02
:101B5100900029E090007BF0E566900058F0E56880
:101B6100900063F0E569900064F0E56A900075F01B
:101B7100E56590007DF0E56790007EF0E5649000FA
:101B810081F0E563900082F090002AE090013BF043
:101B910090002BE090013CF090002CE090013DF092
:101BA100900041E0900091F0900042E0900092F0AE
:101BB100900043E0900093F0900044E0900094F096
:101BC100900045E0900095F0900046E0900096F07E
:101BD100900047E0900097F0900048E0900098F066
:101BE100900033E090009AF0900034E090009BF078
:101BF100900035E090009CF0900036E090009DF060
:101C01007400900083F07441900126F07469900192
:101C110027F07473900128F07469900129F0746EB3
:101C210090012AF0742090012BF0744190012CF066
:101C3100743790012DF0743590012EF074309001BD
:101C41002FF07445900130F07420900131F074351B
:101C5100900132F07453900133F07470900134F0BC
:101C6100900415E0900455F0743A90074FF074FD1C
:101C7100900750F01200C9900004E4F0A3F0900026
:101C8100067475F0A37430F09000087475F0A374B5
:101C910030F0855859D2CA754C00D29C741B900003
:101CA10023F0E556C394065005E551B55203021DD4
:101CB1007FC207E55175F040A4FFAEF090032312F7
:101CC100001EE030E003D38001C39296E55175F028
:101CD10040A4FFAEF090032412001EE030E003D3D5
:101CE1008001C39295E55175F040A4FFAEF09003D9
:101CF1002512001EE030E003D38001C392A0E5511C
:101D010075F040A4FFAEF090032612001EE030E013
:101D110003D38001C3920CE55175F040A4FFAEF0EE
:101D210090032712001EE030E003D38001C3920D1F
:101D3100E556B40206E551640360028002C20DE576
:101D410056B40106E551640260028004D2A0C20DBE
:101D5100E556B4010BE551B40106E560640160028A
:101D61008002C20D855152AE29AF2A7405BE00030F
:101D71009F5007E545D3940550028002D287E5566E
:101D8100D394055003021F0FC207E551D3940150AC
:101D910003021E3DE55175F040A4FFAEF090031F14
:101DA10012001EE0A829B80007D3952A4002155158
:101DB100E55165527003021E3AE55175F040A4FFEA
:101DC100AEF090032312001EE030E003D38001C384
:101DD1009296E55175F040A4FFAEF09003241200F5
:101DE1001EE030E003D38001C39295E55175F040C8
:101DF100A4FFAEF090032512001EE030E003D38073
:101E010001C392A0E55175F040A4FFAEF090032606
:101E110012001EE030E003D38001C3920CE551753E
:101E2100F040A4FFAEF090032712001EE030E00363
:101E3100D38001C3920D855152021F0FE556B4069E
:101E4100419000ADE030E003D38001C39296900051
:101E5100AEE030E003D38001C392959000AFE03053
:101E6100E003D38001C392A09000B0E030E003D33F
:101E71008001C3920C9000B1E030E003D38001C334
:101E8100920DE556B407419000A6E030E003D380FF
:101E910001C392969000A7E030E003D38001C39282
:101EA100959000A8E030E003D38001C392A0900098
:101EB100A9E030E003D38001C3920C9000AAE03086
:101EC100E003D38001C3920DE556B4084190009F11
:101ED100E030E003D38001C392969000A0E030E0AF
:101EE10003D38001C392959000A1E030E003D38039
:101EF10001C392A09000A2E030E003D38001C3921D
:101F01000C9000A3E030E003D38001C3920D900058
:101F110073E06058E54575F00284FF7E0090014F43
:101F210012001EE0F55CE54775F00A84FF7E009023
:101F3100024F12001EE0F55DE55C255DD39464401F
:101F41000BE55C255DC39464F55C8003755C00E57D
:101F51005C75F00284FF7E008F5CEFC39433500701
:101F6100EF24CDF55C8003755CFF801CE54575F0C1
:101F71000284FF7E0090014F12001EE075F0028482
:101F8100FF7E00EF24CDF55CE595C3955C4004C26E
:101F9100938002D293A207B34005E556B4070375B7
:101FA10073CDE595C395734004C2948002D294E544
:101FB1004575F00284FF7E0090018112001EE075DC
:101FC100F00284FF7E00EF24CDF56FE595C3956F98
:101FD1005006A20CB3B340028004D2918002C29198
:101FE100E54575F00284FF7E009001B312001EE00A
:101FF10075F00284FF7E00EF24CDF570E595C39561
:10200100705006A20DB3B340028004D2928002C286
:1020110092E543C394064003022600A2EDB35003A8
:10202100022600C2EDE54360030221777E017F00B5
:10203100E5BE124325E5BD2FFF50010E900000EED5
:10204100F0A3EFF0900029E0B401177E0F7FFF901D
:102051000000E0FCA3E0FD120003900000EEF0A3FD
:10206100EFF090007AE0B4025B900000E0FEA3E0A4
:10207100FF90000AE0FCA3E0FDEDD39FEC9E400F32
:10208100900000E0F8A3E090000AC8F0A3C8F09027
:102091000000E0FEA3E0FF90000CE0FCA3E0FDEFF8
:1020A100D39DEE9C400F900000E0F8A3E090000C5F
:1020B100C8F0A3C8F0900000E0FEA3E0FF74041292
:1020C10043178F4490007AE07060900000E0FEA317
:1020D100E0FF90000AE0FCA3E0FDEFD39DEE9C4001
:1020E1000D120003900000EEF0A3EFF080079000C6
:1020F10000E4F0A3F0900000E0FEA3E0FF741012F2
:102101004325900026E08E048F05FF1243079000BF
:1021110000ECF0A3EDF07400D39D74019C40089095
:102121000001E0F54480037544FFE54475F00AA41D
:10213100FFAEF074198E048F05FF1243078D45ED34
:102141002532FFAE3150010E74011243178F4585C0
:102151004532753100EFD3946240037545629000BA
:1021610073E064016006900067E0600280057543DA
:1021710001800375BB17E543B401028003022232DB
:102181007E017F00E5BE124325E5BD2FFF50010E04
:10219100900000EEF0A3EFF0900073E0B4017CE555
:1021A1003445336025AC33AD341DBDFF011C8F02B6
:1021B1008E038C068D07903FC512002EE493FE74AA
:1021C1000193FFEFC39AEE9B4002800578331243DF
:1021D1004FAE33AF3474B3BE0025D39F402190007E
:1021E10000E0FCA3E0FD0FBF00010E903FC512000F
:1021F1002EE493FE740193FFEDC39FEC9E40028099
:1022010005783312003FAE33AF34E56A12432574CB
:10221100648E048F05FF1243078D47900073E064BD
:10222100026006900067E0600575BB168003754388
:1022310002E543B4020280030223207E017F00E510
:10224100BE124325E5BD2FFF50010E900000EEF0B8
:10225100A3EFF0900073E0B4027EE53445336025CE
:10226100AC33AD341DBDFF011C8F028E038C068D76
:1022710007903E5B12002EE493FE740193FFEFC3BF
:102281009AEE9B40028005783312434FAE33AF3450
:1022910074B3BE0025D39F4021900000E0FCA3E071
:1022A100FD0FBF00010E903E5B12002EE493FE7401
:1022B1000193FFEDC39FEC9E40028005783312002D
:1022C1003FAE33AF34E56A12432574648E048F0543
:1022D100FF1243078D478033900067E0602D900027
:1022E10000E0FEA3E0FFEFD39400EE9408400F90CE
:1022F1000067E0B40104C2098002D209800D900098
:1023010067E0B40104D2098002C209900073E07051
:1023110003754700900067E07002C20975BB1FE5B5
:1023210043B403457E017F00E5BE124325E5BD2F81
:10233100FF50010E900000EEF0A3EFF0740912437C
:102341002574E68E048F05FF1243078C418D42E50B
:102351004A2DFD50010C74018C068D071243178E16
:10236100418F4285424A75BB19E543B4040280039B
:102371000224E87E017F00E5BE124325E5BD2FFF63
:1023810050010E900000EEF0A3EFF0740412431719
:102391008F4BE564B401028003022455756B00750F
:1023A1006B00E56BD394074003022442E56B900078
:1023B1004112433DE0D3954B501AE56B9000411219
:1023C100433DE0F404254BFEE56B90003712433D9D
:1023D100EEF08017E56B90004112433DE0C3954B51
:1023E100FEE56B90003712433DEEF0E56BC39404BC
:1023F1004009900085E0C3956B503BE56B6029E592
:102401006B90003712433DFEE0FFEE90003FE0D3BA
:102411009F4013E56B90003712433DE090003FF081
:10242100E56B900040F0800E900037E090003FF0A7
:102431007400900040F0786B740126F6400302238B
:10244100A3900040E0F4042408F556E556D3940522
:102451004002C287E564D39401402FE54BD3946ECB
:102461004004D20F8002C20F755605E564B402051F
:10247100A20FB340028003755607E564B40306A2B8
:102481000FB3B340028003755607E55765566028C0
:10249100E556B4050DE557D394054006E5516401B1
:1024A1006002800C75510290004E7401F0755A0063
:1024B100855657E55104F552E556B40708E5B5448C
:1024C10020F5B58006E5B554DFF5B5E5566406603F
:1024D10005E556B40808E5B54410F5B58006E5B53F
:1024E10054EFF5B575BB13E543B40502800302252E
:1024F100FC7E017F00E5BE124325E5BD2FFF5001A3
:102501000E900000EEF0A3EFF074041243178F4613
:10251100E563B4020280030225F9756B00756B0057
:10252100E56BD3940340030225B0E56B90003312B1
:10253100433DE0D39546501AE56B90003312433D7D
:10254100E0F4042546FEE56B90002D12433DEEF0CC
:102551008017E56B90003312433DE0C39546FEE5DD
:102561006B90002D12433DEEF0E56B6029E56B9019
:10257100002D12433DFEE0FFEE900031E0D39F407D
:1025810013E56B90002D12433DE0900031F0E56BB7
:10259100900032F0800E90002DE0900031F0740038
:1025A100900032F0786B740126F6400302252190E9
:1025B1000083E07043E52A45296036E558C394035A
:1025C100500A900032E004C3940340028007900057
:1025D10032E004F558E558D39402400A900032E005
:1025E10004D3940250028007900032E004F5588031
:1025F10007900032E004F55875BB180543D2ECE5AD
:102601005ED39404500302279A75CF01C293AE356D
:10261100AF367488D39F74139E4005A2A5B34014AE
:10262100AE35AF367488D39F74139E4005A2A4B310
:1026310040028048783512003FAE35AF36EFB4889E
:102641003BEEB41337A2A5B35009900050E0D395E7
:10265100515002800405518011A2A5B35008900089
:1026610050E0655160028002D207A2A4B35007E591
:1026710051D39401500280041551C207A2A5B3B3EE
:102681005006A2A4B3B3400280067536007535002A
:10269100E5516552700302271CE55175F040A4FF16
:1026A100AEF090032312001EE030E003D38001C39B
:1026B1009296E55175F040A4FFAEF090032412000C
:1026C1001EE030E003D38001C39295E55175F040DF
:1026D100A4FFAEF090032512001EE030E003D3808A
:1026E10001C392A0E55175F040A4FFAEF09003261E
:1026F10012001EE030E003D38001C3920CE5517556
:10270100F040A4FFAEF090032712001EE030E0037A
:10271100D38001C3920DC294855152A20740057521
:1027210073CD80037573FFE595C395734004C2941F
:102731008002D294E54575F00284FF7E009001810C
:1027410012001EE075F00284FF7E00EF24CDF56FCC
:10275100E595C3956F5006A20CB3B340028004D235
:10276100918002C291E54575F00284FF7E009001DF
:10277100B312001EE075F00284FF7E00EF24CDF558
:1027810070E595C395705006A20DB3B34002800465
:10279100D2928002C29202260AAE25AF26EFD394CE
:1027A10020EE944E50030228A11204ABC28E758D07
:1027B10000758B00754C00D28EC207757200757161
:1027C100007573CD7551057524007523007554008E
:1027D100755A00E5B554BFF5B590005AE06008E5BB
:1027E100B54480F5B58006E5B5547FF5B590004A4E
:1027F100E0B40104D2A18002C2A1900049E0B40179
:1028010004D2A28002C2A2A209B34004D2978002DC
:10281100C29790006CE0601812397AA200B34008A8
:10282100E5B54408F5B58006E5B554F7F5B5800280
:10283100C20090006FE06018123ACFA202B34008C4
:10284100E5B54402F5B58006E5B554FDF5B580065C
:10285100E5B554FDF5B590000E74FDF0A374E8F0F4
:10286100E543B40603754300900025E4F0752600A6
:10287100752500758D00758B00754C00900024E066
:10288100C394035008900024E004F0800674039080
:102891000024F0900024E0B40306E5B554FEF5B53C
:1028A100AE27AF28EFD39410EE9427401CC2CA750F
:1028B100CD0075CC00752800752700D2CA754E0071
:0C28C100752A00752900755500020CE313
:103C81000000010001320164019601960200021256
:103C910002240200020003000340038003C0040069
:103CA1000440048004C0050006000600060006006A
:103CB100060006000600060000FF013101630195C0
:103CC10001FF01FF0211022302FF02FF02FF033F76
:103CD100037F03BF03FF043F047F04BF04FF05FF0D
:103CE10006FF06FF06FF06FF06FF06FF06FF06FFAB
:103CF1000FAA0FA50F9F0F9A0F940F8D0F870F809B
:103D01000F780F710F680F600F570F4E0F450F3B64
:103D11000F300F250F1A0F0E0F020EF50EE80EDBF6
:103D21000ECC0EBE0EAE0E9F0E8E0E7D0E6C0E5A7A
:103D31000E470E340E200E0C0DF70DE20DCB0DB516
:103D41000D9D0D850D6D0D540D3A0D200D050CE9E0
:103D51000CCE0CB10C940C760C580C3A0C1B0BFBD2
:103D61000BDB0BBB0B9A0B790B570B350B130AF1C2
:103D71000ACE0AAB0A870A640A400A1C09F809D468
:103D810009B0098C09670943091F08FB08D608B265
:103D9100088E086A0846082307FF07DC07B907965B
:103DA10007730751072F070D06EC06CA06AA0689F5
:103DB10006690649062A060A05EC05CD05B00592F5
:103DC10005750558053C0520050504EA04CF04B531
:103DD100049C04820469045104390422040B03F491
:103DE10003DE03C803B2039D038903750361034D19
:103DF100033B03280316030402F202E102D102C0CD
:103E010002B002A0029102820273026502570249C6
:103E1100023C022F02220216020901FD01F201E613
:103E210001DB01D001C601BB01B101A7019D0194D4
:103E3100018B018201790170016801600158015013
:103E41000148014101390132012B0125011E0118EF
:103E51000111010B010500FF00FA0FA60FA00F9938
:103E61000F920F8B0F840F7C0F740F6B0F620F5823
:103E71000F4E0F430F380F2C0F1F0F120F050EF7A8
:103E81000EE80ED80EC80EB70EA50E930E800E6C5E
:103E91000E580E420E2C0E150DFD0DE40DCB0DB17D
:103EA1000D950D790D5D0D3F0D200D010CE10CC03F
:103EB1000C9E0C7C0C590C350C100BEA0BC40B9EA0
:103EC1000B760B4F0B260AFD0AD40AAA0A800A5563
:103ED1000A2A09FF09D409A8097C0950092508F90A
:103EE10008CD08A10875084A081E07F307C8079DF1
:103EF10007730749072006F706CE06A6067E065772
:103F01000630060A05E405BF059B05770554053211
:103F1100051004EF04CE04AE048F0471045304357C
:103F2100041903FD03E203C703AD0394037B036399
:103F3100034B0334031E030802F302DE02CA02B676
:103F410002A30291027F026D025C024C023C022C30
:103F5100021D020E020001F201E401D701CA01BEF5
:103F610001B101A6019A018F0185017A01700166F3
:103F7100015D0153014A0141013901310129012149
:103F810001190112010B010400FD00F700F000EA24
:103F910000E400DE00D900D300CE00C900C400BF98
:103FA10000BA00B500B100AD00A800A400A0009CBB
:103FB100009900950091008E008A0087008400819D
:043FC100007E007B03
:1028EE00751A00751900AE19AF1AAC17AD18EDC3F5
:1028FE009FEC9E401674FF1242F775CF01781A7442
:10290E000126F6500418E436F650DB22900787E4D1
:10291E00F0A3F0751000750F00751300751400C24A
:10292E0010D21122C2AF75D900758F0375B7A57578
:10293E00B7F190F800E4F0758F0175B7A575B7F192
:10294E00E50890F800F075B7A575B7F190F801E4B9
:10295E00F075B7A575B7F190079EE090F802F07587
:10296E00B7A575B7F19007A2E090F803F075B7A57B
:10297E0075B7F190079FE090F804F075B7A575B79D
:10298E00F19007A0E090F805F075B7A575B7F19036
:10299E0007A1E090F806F075B7A575B7F19007A3FB
:1029AE00E090F807F0758F0075D940D2AF229007EE
:1029BE0089E0B4AB61C2AF75D90075B62275F52248
:1029CE00758F0375B7A575B7F1740090F600F075A5
:1029DE008F01750A00750900AE09AF0A7413BE00A7
:1029EE00279F402475B7A575B7F190078A12001E70
:1029FE00E0FC90F60012001EECF0780A740126F648
:102A0E00500418E436F650D0758F0075F51175B672
:102A1E002075D940D2AF22C2AF75D90075F5227597
:102A2E000A00750900AE09AF0A7413BE00229F405A
:102A3E001F90F60012001EE493FC90078A12001EEF
:102A4E00ECF0780A740126F6500418E436F650D5E8
:102A5E0075F51175D940D2AF22900789E0B4AA025C
:102A6E008003022BA4C2AF75D90075B62275F5226C
:102A7E00758F0375B7A575B7F1740090EE00F075FC
:102A8E00B7A575B7F1740090F000F075B7A575B7DE
:102A9E00F1740090F200F075B7A575B7F17400905F
:102AAE00F400F0758F01750A00750900AE09AF0AC2
:102ABE0074FFC39F74019E402475B7A575B7F1903E
:102ACE00004F12001EE0FC90EE0012001EECF0789B
:102ADE000A740126F6500418E436F650CF750A0033
:102AEE00750900AE09AF0A74FFC39F74019E40249E
:102AFE0075B7A575B7F190024F12001EE0FC90F06D
:102B0E000012001EECF0780A740126F6500418E448
:102B1E0036F650CF750A00750900AE09AF0A74FF7C
:102B2E00C39F74019E402475B7A575B7F190044FED
:102B3E0012001EE0FC90F20012001EECF0780A74F7
:102B4E000126F6500418E436F650CF750A007509C2
:102B5E0000AE09AF0A74FFC39F74019E402475B77F
:102B6E00A575B7F190064F12001EE0FC90F400120E
:102B7E00001EECF0780A740126F6500418E436F6BE
:102B8E0050CF758F0075F51175B62075D940D2AF3F
:102B9E00743A90074FF022900789E0B4AA0280039E
:102BAE00022CE2C2AF75D90075B62275F522758F6B
:102BBE000375B7A575B7F1740090E600F075B7A56B
:102BCE0075B7F1740090E800F075B7A575B7F1749C
:102BDE000090EA00F075B7A575B7F1740090EC009F
:102BEE00F0758F01750A00750900AE09AF0A74FF02
:102BFE00C39F74019E402475B7A575B7F190004F21
:102C0E0012001EE0FC90E60012001EECF0780A7432
:102C1E000126F6500418E436F650CF750A007509F1
:102C2E0000AE09AF0A74FFC39F74019E402475B7AE
:102C3E00A575B7F190024F12001EE0FC90E800124D
:102C4E00001EECF0780A740126F6500418E436F6ED
:102C5E0050CF750A00750900AE09AF0A74FFC39F05
:102C6E0074019E402475B7A575B7F190044F1200FC
:102C7E001EE0FC90EA0012001EECF0780A740126A9
:102C8E00F6500418E436F650CF750A00750900AEFA
:102C9E0009AF0A74FFC39F74019E402475B7A575D2
:102CAE00B7F190064F12001EE0FC90EC0012001ED1
:102CBE00ECF0780A740126F6500418E436F650CF7C
:102CCE00758F0075F51175B62075D940D2AF743A6F
:102CDE0090074FF022900789E0B4AA028003022EDB
:102CEE0020C2AF75D90075B62275F522758F0375A2
:102CFE00B7A575B7F1740090DE00F075B7A575B77E
:102D0E00F1740090E000F075B7A575B7F1740090FE
:102D1E00E200F075B7A575B7F1740090E400F07598
:102D2E008F01750A00750900AE09AF0A74FFC39FC3
:102D3E0074019E402475B7A575B7F190004F12002F
:102D4E001EE0FC90DE0012001EECF0780A740126E4
:102D5E00F6500418E436F650CF750A00750900AE29
:102D6E0009AF0A74FFC39F74019E402475B7A57501
:102D7E00B7F190024F12001EE0FC90E00012001E10
:102D8E00ECF0780A740126F6500418E436F650CFAB
:102D9E00750A00750900AE09AF0A74FFC39F74016E
:102DAE009E402475B7A575B7F190044F12001EE032
:102DBE00FC90E20012001EECF0780A740126F65028
:102DCE000418E436F650CF750A00750900AE09AF47
:102DDE000A74FFC39F74019E402475B7A575B7F1A1
:102DEE0090064F12001EE0FC90E40012001EECF064
:102DFE00780A740126F6500418E436F650CF758F13
:102E0E000075F51175B62075D940D2AF743A90079A
:102E1E004FF022900789E0B4AA028003022F5EC20F
:102E2E00AF75D90075B62275F522758F0375B7A5E6
:102E3E0075B7F1740090D600F075B7A575B7F1743B
:102E4E000090D800F075B7A575B7F1740090DA0050
:102E5E00F075B7A575B7F1740090DC00F0758F01B1
:102E6E00750A00750900AE09AF0A74FFC39F74019D
:102E7E009E402475B7A575B7F190004F12001EE065
:102E8E00FC90D60012001EECF0780A740126F65063
:102E9E000418E436F650CF750A00750900AE09AF76
:102EAE000A74FFC39F74019E402475B7A575B7F1D0
:102EBE0090024F12001EE0FC90D80012001EECF0A3
:102ECE00780A740126F6500418E436F650CF750AC7
:102EDE0000750900AE09AF0A74FFC39F74019E40CE
:102EEE002475B7A575B7F190044F12001EE0FC9043
:102EFE00DA0012001EECF0780A740126F65004185F
:102F0E00E436F650CF750A00750900AE09AF0A74A3
:102F1E00FFC39F74019E402475B7A575B7F1900647
:102F2E004F12001EE0FC90DC0012001EECF0780A3E
:102F3E00740126F6500418E436F650CF758F0075DE
:102F4E00F51175B62075D940D2AF743A90074FF08F
:102F5E0022C2AF75D90075F522750A00750900AE4B
:102F6E0009AF0A74FFC39F74019E401F90EE0012BA
:102F7E00001EE493FC90004F12001EECF0780A74D1
:102F8E000126F6500418E436F650D4750A00750979
:102F9E0000AE09AF0A74FFC39F74019E401F90F0EC
:102FAE000012001EE493FC90024F12001EECF0780B
:102FBE000A740126F6500418E436F650D4750A0049
:102FCE00750900AE09AF0A74FFC39F74019E401FBE
:102FDE0090F20012001EE493FC90044F12001EECBF
:102FEE00F0780A740126F6500418E436F650D475BB
:102FFE000A00750900AE09AF0A74FFC39F74019EE3
:10300E00401F90F40012001EE493FC90064F120035
:10301E001EECF0780A740126F6500418E436F650C9
:10302E00D475F51175D940D2AF22C2AF75D90075DE
:10303E00F522750A00750900AE09AF0A74FFC39F29
:10304E0074019E401F90E60012001EE493FC900057
:10305E004F12001EECF0780A740126F6500418E4A4
:10306E0036F650D4750A00750900AE09AF0A74FF22
:10307E00C39F74019E401F90E80012001EE493FC53
:10308E0090024F12001EECF0780A740126F65004DE
:10309E0018E436F650D4750A00750900AE09AF0A69
:1030AE0074FFC39F74019E401F90EA0012001EE43D
:1030BE0093FC90044F12001EECF0780A740126F671
:1030CE00500418E436F650D4750A00750900AE099E
:1030DE00AF0A74FFC39F74019E401F90EC00120054
:1030EE001EE493FC90064F12001EECF0780A740159
:1030FE0026F6500418E436F650D475F51175D940FD
:10310E00D2AF22C2AF75D90075F522750A007509C6
:10311E0000AE09AF0A74FFC39F74019E401F90DE7C
:10312E000012001EE493FC90004F12001EECF0788B
:10313E000A740126F6500418E436F650D4750A00C7
:10314E00750900AE09AF0A74FFC39F74019E401F3C
:10315E0090E00012001EE493FC90024F12001EEC51
:10316E00F0780A740126F6500418E436F650D47539
:10317E000A00750900AE09AF0A74FFC39F74019E61
:10318E00401F90E20012001EE493FC90044F1200C8
:10319E001EECF0780A740126F6500418E436F65048
:1031AE00D4750A00750900AE09AF0A74FFC39F7487
:1031BE00019E401F90E40012001EE493FC90064F07
:1031CE0012001EECF0780A740126F6500418E4364C
:1031DE00F650D475F51175D940D2AF22C2AF75D95C
:1031EE000075F522750A00750900AE09AF0A74FF65
:1031FE00C39F74019E401F90D60012001EE493FCE4
:10320E0090004F12001EECF0780A740126F650045E
:10321E0018E436F650D4750A00750900AE09AF0AE7
:10322E0074FFC39F74019E401F90D80012001EE4CD
:10323E0093FC90024F12001EECF0780A740126F6F1
:10324E00500418E436F650D4750A00750900AE091C
:10325E00AF0A74FFC39F74019E401F90DA001200E4
:10326E001EE493FC90044F12001EECF0780A7401D9
:10327E0026F6500418E436F650D4750A0075090087
:10328E00AE09AF0A74FFC39F74019E401F90DC000D
:10329E0012001EE493FC90064F12001EECF0780A0A
:1032AE00740126F6500418E436F650D475F51175EF
:1032BE00D940D2AF22E51464046006E59964FF603C
:1032CE00028031A2104004D2108027E514600874E9
:1032DE00E62514900023F0E513600874F025139092
:1032EE000023F0E514B4010280FE7514007513007E
:1032FE00C2108002C210E514903C24F82828737581
:10330E001400E599B4FF03751301E599B4FE037536
:10331E001302E599B4FD03751303E599B4FC037527
:10332E001304E599B4FA03751305E599B4FB067514
:10333E0014011204ABE599B4F9067514041204AB2A
:10334E00E599D394E54007E599C394F040028016C1
:10335E008599157514027E017F00E515C394E6125A
:10336E0043258E0D8F0E900787E4F0A3F0E599D3D9
:10337E0094C44007E599C394E640028028859915C8
:10338E0075140374E5C39515F50E750D00AE0DAFEE
:10339E000E903C8112002EE493F8740193900787EF
:1033AE00C8F0A3C8F0D299023838900787E0FEA380
:1033BE00E0FFEFC39400EE94054009EFD394FFEEC7
:1033CE0094064013900787E0FEA3E0FF90004F1293
:1033DE00001EE599F0800385996C90078712000E08
:1033EE00900787E0FEA3E0FFEFB40106EEB40702FC
:1033FE00800302364590074FE0B43C02800302364C
:10340E004575FFA0A20AB35005A20BB340030235C7
:10341E0038C29C90007BE090078DF0900058E090B1
:10342E00078EF0900063E090078FF0900064E090BC
:10343E000790F0900075E0900791F090007DE0907D
:10344E000792F090007EE0900793F0900081E0905C
:10345E000794F0900082E0900795F090013BE09089
:10346E000796F090013CE0900797F090013DE090B8
:10347E000798F0900091E0900799F0900092E090FC
:10348E00079AF0900093E090079BF0900094E090E4
:10349E00079CF0900095E090079DF0900096E090CC
:1034AE00079EF0900097E090079FF0900098E090B4
:1034BE0007A0F090009AE09007A1F090009BE0909A
:1034CE0007A2F090009CE09007A3F090009DE09082
:1034DE0007A4F07400900083F01200C974AB90073B
:0D34EE0089F01229BC74AA900789F0E558F6
:063C240002330D0233B86B
:1034FB00903C45F82828738012122A67800D122BF6
:0B350B00A58008122CE38003122E2183
:0F3C450002350202350402350902350E0235132D
:10351600900789E4F090013BE0700C90013CE0706C
:103526000690013DE060028004C20A8002D20A02CF
:10353600363AC29C900079E090078AF090005FE0EE
:1035460090078BF0900060E090078CF090007BE095
:1035560090078DF0900058E090078EF0900063E0A1
:1035660090078FF0900064E0900790F0900075E06F
:10357600900791F090007DE0900792F090007EE039
:10358600900793F0900081E0900794F0900082E01D
:10359600900795F090013BE0900796F090013CE093
:1035A600900797F090013DE0900798F0900091E029
:1035B600900799F0900092E090079AF0900093E0BF
:1035C60090079BF0900094E090079CF0900095E0A7
:1035D60090079DF0900096E090079EF0900097E08F
:1035E60090079FF0900098E09007A0F090009AE076
:1035F6009007A1F090009BE09007A2F090009CE05D
:103606009007A3F090009DE09007A4F0740090004E
:1036160083F074AB900789F01229BC74AA900789CD
:10362600F0122A67122BA5122CE3122E21D29C75BA
:1036360099FB80FED29C7514007513007599FB02E8
:103646003838900787E0FEA3E0FFEF4E70068599B5
:1036560010750F00900787E0FEA3E0FF74016F4E20
:10366600701BAC0FAD10AA0DAB0EED2BFBEC3AFAAE
:103676008A068B0790004F12001EE599F090078787
:1036860012000E900787E0FEA3E0FF74026F4E70F3
:103696000C1200C985159975140075130002383887
:1036A600900787E0FEA3E0FF90004F12001EE59909
:1036B600F090078712000E900787E0FEA3E0FFACAC
:1036C6000DAD0E8F028E038C068D07903CB912004D
:1036D6002EE493F9740193FEEAD39EEB9940098593
:1036E6001599751400751300023838900787E0FEA7
:1036F600A3E0FF90004F12001EE599F09007871295
:10370600000E900787E0FEA3E0FFEFB40006EEB4DC
:103716000102800302383875FFA090001CE0D394A4
:10372600C7400B90001CE0C394C8F516801A9000A1
:103736001CE0D39463400B90001CE0C39464F51620
:10374600800690001CE0F516E51675F002A4FFAEA3
:10375600F08F6BEF90004F12433DEFFCE0FDEC90D5
:10376600005212433DEDFCE0FDEC2DB51602800340
:1037760002382A0FEF90004F12433DE56BFFE0FC45
:10378600EF90005312433DECFFE0FCEFC39CB516EF
:1037960002800302382AE56B90005112433DE56B27
:1037A600FFE0FCEF90005412433DECFFE0FCEF2CF1
:1037B600B51671E56B90005512433DE0C395169022
:1037C600079EF0E56B90005612433DE0C3951690B8
:1037D600079FF0E56B90005912433DE0C3951690A4
:1037E60007A0F0E56B90005A12433DE0C395169092
:1037F60007A1F0E56B90005B12433DE0C395169080
:1038060007A2F0E56B90005C12433DE0C39516906D
:1038160007A3F01229327599F97518647517001205
:1038260028EE80FE7599FF7518647517001228EE4C
:0238360080FE12
:093C2A000236480236A60236F10A
:1038380022E513903C33F8282873023979900787DA
:10384800E0FEA3E0FF90001212001EE0F599900739
:103858008712000E900787E0FEA3E0FF74116F4EF9
:1038680070037513000239798562990239799007D6
:1038780087E0FEA3E0FF90004F12001EE0F599EFED
:10388800B40107EEB4070375130090078712000E02
:07389800023979900788E076
:0F3C330002384202384502387002387602389B58
:10389F00903C54F828287385249902396E852A990B
:1038AF0002396E85449902396E85479902396E85C2
:1038BF00519902396E85609902396E855699023990
:1038CF006E85589902396E756E0090006AE0700629
:1038DF00900069E060028016A2A44006E56E4404E1
:1038EF00F56EA2A54006E56E4402F56E801A9000B3
:1038FF004AE0B40106E56E4410F56E900049E0B45D
:10390F000106E56E4420F56EA207B34006E56E444E
:10391F0001F56EA209B34006E56E4408F56E856E9B
:10392F0099803CA211B340077599FAC2118017A272
:10393F000EB3400575990F800B900023E0F5999019
:10394F000023E4F0C20E80178542998012854B99AF
:0F395F00800D85469980087599FC8003751300CB
:103C54000238A60238AC0238B20238B80238BE02C2
:103C640038C40238CA0238D00238D602393202398E
:0D3C74005702395C02396102396602396B72
:0B396E0090078712000E800312004833
:033C4200023976CE
:103979002290006CE0B4010385241190006CE0B43E
:103989000203852A1190006CE0B403038544119069
:10399900006CE0B4040385471190006CE0B40503A2
:1039A90085511190006CE0B4060385561190006CA6
:1039B900E0B4070385581190006DE0FE90006EE0B9
:1039C900C39E5003023A5090006CE0D39404402CFB
:1039D90090006DE0D39511500990006EE0C39511E8
:1039E90050028002D20090006DE0D39511500990E9
:1039F900006EE0C395115002C200804990006CE04E
:103A0900B4041890006EE0C395115002D2009000E2
:103A19006DE0D395114002C200802A90006DE0C389
:103A29009511500990006EE0D3951150028002D291
:103A39000090006DE0D39511500990006EE0C39598
:103A4900115002C200807E90006CE0D39404402C97
:103A590090006DE0C39511400990006EE0D3951177
:103A690040028002C20090006DE0C39511400990A8
:103A7900006EE0D395114002D200804990006CE0BD
:103A8900B4041890006DE0C395115002C200900073
:103A99006EE0D395114002D200802A90006DE0C3F8
:103AA9009511400990006EE0D395114002D2009023
:103AB900006DE0D39511400990006EE0C395114067
:103AC900028002C2002290006FE0B4010385241134
:103AD90090006FE0B40203852A1190006FE0B403EF
:103AE9000385441190006FE0B404038547119000E9
:103AF9006FE0B4050385511190006FE0B4060385AA
:103B0900561190006FE0B40703855811900070E0DA
:103B1900FE900071E0C39E5003023BA590006FE048
:103B2900D39404402C900070E0D395115009900073
:103B390071E0C3951150028002D202900070E0D367
:103B490095115009900071E0C395115002C202808D
:103B59004990006FE0B40418900071E0C3951150CA
:103B690002D202900070E0D395114002C202802A6D
:103B7900900070E0C395115009900071E0D3951140
:103B890050028002D202900070E0D3951150099042
:103B99000071E0C395115002C202807E90006FE06F
:103BA900D39404402C900070E0C395114009900013
:103BB90071E0D3951140028002C202900070E0C307
:103BC90095114009900071E0D395114002D202800D
:103BD9004990006FE0B40418900070E0C39511504B
:103BE90002C202900071E0D395114002D202802AEC
:103BF900900070E0C395114009900071E0D39511D0
:103C09004002D202900070E0D395114009900071F2
:0B3C1900E0C3951140028002C20222AD
:09433D002582F58250020583225D
:10002E00EF2F500205832582F582E5833E2EF58360
:01003E00229F
:08000300C3EF9DFFEE9CFE22FD
:08003F000806B60002180622B3
:0D000E00A3E004F07006124333E004F0227A
:08434F000816B6FF0218162241
:0E431700048007C3CE13CECF13CFD5E0F6221D
:1041C500BC000FBE0008ED8FF084FFADF022E4FEC9
:1041D500FF22BE000DEF60FE54F0606F20E7030282
:1041E500427BEAC0E0EBC0E078017A0075F001EEB1
:1041F50020E710EF25E0FFEE33FE0AC5F023C5F0FA
:1042050030E7F0EA5407F9096A7A007B0060010893
:10421500C3EC9E40167004ED9F4010ED9FFDEC9E93
:10422500FCE5F0CA4ACA03F5F08005E5F003F5F0B0
:10423500C3EE13FEEF13FFD9D77908CACBCAD8D07E
:10424500EAFEEBFFD0E0FBD0E0FA22EC8FF084FC35
:10425500ED54F045F0C48FF084FEEDC454F045F004
:10426500C48FF084FDEEC4FE54F02DFFEE540F3CD8
:10427500FEADF07C0022790078008FF0EC7E0820FE
:10428500E70DC3CD33CD33C933C9C833C8DEF08498
:1042950049F9E5F08FF0BE00E6FD7C00E9FFE8FE98
:0142A50022F6
:0E432500F88FF0A4FFE5F0CE88F0A42EFE2263
:1042F700600D782B024301007830D8FED5E0F82214
:10430700EEC0E07E001241C5EFFDEEFCD0E0FE22DC
:03000B000242A608
:03001B000242C1DD
:03002B000242DCB2
:0300000002434672
:0943460075817475D00002082392
:0B001E00E5822FF582E5833EF583228A
:0A4333000582D5820215831582224F
:1042A600C0E0C0F0C083C082C0D075D0001208182C
:1042B600D0D0D082D083D0F0D0E032C0E0C0F0C001
:1042C60083C082C0D075D00012081BD0D0D082D057
:1042D60083D0F0D0E032C0E0C0F0C083C082C0D04E
:1042E60075D00012081ED0D0D082D083D0F0D0E096
:0142F6003295
:00000001FF
